:020000040000FA
:060000000219FD020310CD
:03001300020501E2
:03001B0002008D53
:03002B000202D5F9
:03005B000205108B
:030073000202FD89
:100080000406080C10182030406080A0C0C2AFC227
:10009000A853E6EFC28E856B8BC0D0D2D3C0E0C030
:1000A000F0C2CAA8CCA9CDD2CAD2AF758A00C3E823
:1000B000956CF8E9956DF9C3E913F9E813F8E5666D
:1000C0006007C3E913F9E813F8E97025E8956E4075
:1000D00020956E501CE582B410177C007B007A00DE
:1000E0007908900000A86AE5667004C3E813F80177
:1000F000FA900000D2A8D2AA61BAE0FDC39CC398CE
:1001000040EF98EB33FB0582E0FCC39DC39840E1D0
:1001100098EB33FB0582E0FDC39CC39840D398EB7A
:1001200033FB0582E0FCC39DC39840C598EB33FBCD
:100130000582E0FDC39CC39840B798EB33FB058272
:10014000E0FCC39DC39840A998EB33FB0582E0FD1A
:10015000C39CC398409B98EB33FB0582E0FCC39D96
:10016000C398408D98EB33FB05822175900000D237
:10017000A8D2AA61BAE0FDC39CC39840EF98EA33C5
:10018000FA0582E0FCC39DC39840E198EA33FA0582
:1001900082E0FDC39CC39840D398EA33FA0582E01D
:1001A000FCC39DC39840C598EA33FA0582E0FDC3BD
:1001B0009CC39840B798EA33FA0582E0FCC39DC31C
:1001C0009840A998EA33FA0582E0FDC39CC39840A1
:1001D0009B98EA33FA0582E0FCC39DC398408D9852
:1001E000EA33FA0582EBC46B6A54F0F9EAC454F0BE
:1001F000C3996009900000D2A8D2AA61BAEBF4C4F6
:1002000054F0F9EAF4C4540F49FAEBF4C4540FFB68
:10021000C3EAF99460FAEB9400FB5020C3E97B0039
:100220007A0079006016C3135006F9C39552600A2C
:10023000E9F552755300790080020553303A27C31F
:10024000EA94D0F8EB9407F9400BE8FAE9FB203583
:1002500009D235415A303502C235203902B235C390
:10026000EA33FAEB33FBEB2B3B3BF9C3EB13FBEA33
:1002700013FAEA29FAEB3400FB30E3047AFF7BFF40
:10028000E5255403601B202A18E55D33F9EB700760
:10029000C3E99A4002E9FAE53CC4332AFAEB340098
:1002A000FBC3EA33C4540FF8EB33C454F048F8707E
:1002B00005EA60027801C3EB13FBEA13FA90000031
:1002C000D2A8D2AAE52260021522819E900000D217
:1002D000A8D2AA61BAC0D0C0E0C2CF0541E5236070
:1002E000021523C3E554600575550041F8E5552412
:1002F00001F55550037555FFD0E0D0D032C2AF5351
:10030000E67F7592FA7593FFC22053917FD2AF3288
:10031000C0E0E58A303408856B8BF0A3D0E032D0A2
:10032000E0C2AF53E6EFC0D0C0E0C0F0D2D3D2AF4E
:100330005388EFA88AA98C758A00758C00438810B1
:1003400030331FE8C4540FFAE9C454F04AFAC31317
:100350002AFAC3E833F8E933F9E82AFAE93403FB67
:1003600061AB30320FC3E833E933FAE82AFAE934F3
:1003700000FB61AB303115E875F056A4AAF0E975C1
:10038000F056A42AFAC5F03400FB61ABE875F02BF7
:10039000A4AAF0E975F02BA42AFAC5F03400C3131F
:1003A000FBEA13FAC3EB13FBEA13FAC3EB9409500D
:1003B00009C3EA949AEB940350160522E5227002D1
:1003C0001522C3E5229432500281F475540081F75E
:1003D000E522600215223036067C007D0461EAAC1D
:1003E00031AD32303A04AC33AD34C3EA9CFAEB9D04
:1003F000FB9208AE60AF61303A425007203509D217
:10040000358108303502C235303504AE62AF632025
:100410003902B235C3EA33FAEB33FBA208500AEAD9
:10042000F42401FAEBF43400FBC3EA9428FAEB94C9
:1004300000FB501478007A007B008148A208500825
:1004400078007A007B00819EE52554036019202AFC
:1004500016E55DF9EB7007C3E99A4002E9FAE53C5D
:10046000C42AFAEB3400FBEA8EF0A4F9AAF0EB8E72
:10047000F0A42AFAC5F03400FBC3EB13FDEA13F82D
:100480000FEF146004C3E833F8C3E933EA33FAEB3F
:1004900033FBDFEDEB30E20678FF7AFF7B03885415
:1004A000D230E86003755500C3E55BFC955C400203
:1004B000AC5CC3EC95545008EC75F004A4FAABF0B6
:1004C000EAF4F8EBF45403F98856895775230AE5E2
:1004D0005A30E110D0F0D0E0D0D053F7DF43F740EE
:1004E00043E61032D0F0D0E0D0D053D8FE43DA014A
:1004F00043E6103275230AD0F0D0E0D0D043E610A6
:1005000032C2AAD28EC2CA85CC6C85CD6DD2CA3217
:10051000C2AFC0D0C0E0D2D38556FB8557FC85570B
:100520005A53F7BF53DAFED2A8303402D2AA53E6A8
:10053000EF53F7DF53D8FED0E0D0D0D2AF327901FD
:10054000801479038010790A800C791E8008796400
:10055000800479C880007817E4D5E0FDD8FAD9F690
:100560002278FF20282879A1E76023E548601F74DE
:10057000FF8548F084853FF030290375F005A4F825
:10058000C5F0600278FFC3E8955D5002A85D885C05
:1005900022C3E54794E4E5489400E55C500314A1C8
:1005A000A2046002F55C2275E89022055EC3E55E58
:1005B0009408405330EDF4A8BDA9BE755E00E9FA79
:1005C00079A0E76041EA7006E55F6018800CC3E837
:1005D000955F600EE55F5005600A1480070460FABD
:1005E0008002E55FF55FC39569401B755BC0C394EE
:1005F000044013755B80C39404400B755B40C39447
:10060000044003755B0022E55B2410500274FFF583
:100610005B22743279A687F0A4C5F0A2F733F55DAA
:10062000227547007548F022C2AFC2CAA8CCA9CD36
:10063000AA4130CF010AD2CAD2AFAB42AC43884202
:100640008943C3E89BF8E99C202808F9302C02E193
:1006500038C191AD448A44F9EA9DFA600678FF7981
:10066000FFC176AE45AF468B458C46A842A943C331
:10067000E89EF8E99FF9C3E54813FBE54713FAE85C
:100680002AF547E93BF54850067547FF7548FFC115
:10069000DEAA47AB48AC47AD487E047F02C3EB946B
:1006A00004400D1E1FC3EB940840052029021E1FA5
:1006B000C3ED13FDEC13FCDEF7C3EA9CFAEB9DFBE4
:1006C000EF6009C3E913F9E813F8DFF7EA28FAEB5A
:1006D00039FB8A478B4850067BFF8B478B48C3EB1F
:1006E00094025002D22C3028047F03E1097892E66C
:1006F000FFC3E53D948240110FC3E53D94A0400146
:100700000FC3EF940640027F057E02E548C4540FF4
:10071000F9E548C454F0F8E547C4540F28F8C3E895
:100720009EFAE99400FB4009C3EA9401EB9400505F
:10073000047A01E4FB020784AA47AB48EBC4FEEA53
:10074000C4540F4EFCC3EA9CFAEB9400FBC3E813BD
:10075000C313F8EA28FAEB3400FB8A478B48C3EB53
:1007600094024002C22C7802EBC4FE7B00EAC4541F
:100770000F4EFAC3EA98FA4005C3940150027A0179
:100780007892E6FF302002E184854E92854F93D225
:100790002043E680C3E49AF8E49BF9302C03020876
:1007A00012E8FAE9FBD3E913FDE813FC884E894F00
:1007B000C3EF94036038EF20E00CE82CF8E93DF932
:1007C000ECFAEDFB8013E828F8E939F9C3E82401D5
:1007D000F8E93400F97AFF7BFFC3EF9403400F8AF6
:1007E000508B51884A894B8C4C8D4D02084788505C
:1007F00089518A4A8B4B8C4C8D4D3028127550F0A4
:100800007551FF754CF0754DFF754EF0754FFF0239
:100810000847E8FAD3E813FC884EC3EF940360213D
:10082000EF20E007E82CF8ECFA0132E8282401F880
:100830007AFFC3EF940340098A50884A8C4C02081F
:100840004788508A4A8C4C3020020147753A02D2C0
:100850002043E680E52554036034A847A948C3E94E
:1008600013F9E813F8C3E913F9E813F8302804E999
:100870002440F9C2AF53E67F759100C3E498F59424
:10088000E499F595759104D22043E680D2AF22D247
:1008900021754900752000302B0375204001ADD231
:1008A00021754900752040302B03752000780179AF
:1008B00001202C20E52554036002C2217914E5486B
:1008C000C313700104F8C394144002781430280450
:1008D000781B791B202010E549600C302803D53A9D
:1008E00004D2222154114F0549E59B5440B5200202
:1008F000213E30280908C3E89940011801D420217D
:100900000A08C3E899400201AD01D4C22153E67F31
:10091000759100302C117594007595F8759104D27D
:100920002043E6800208ADE5487EFFC3334005C39F
:10093000334001FEC3E49E759400F595211CC3E588
:10094000399401500201AD30210201ADD80221528B
:1009500001D4C222C2AF53E67F75910085509485C1
:100960005195759104854A92854B93D22043E68038
:10097000D2AFE525540360072029020539801030E5
:10098000220D202B0A2021071581158102139122A7
:1009900078003021027801E53D75F007A4F9E5F013
:1009A00028F5F0E9A2F013A2F113A2F213F53DC36A
:1009B00094785003753D78C3E53D953E400653F26B
:1009C0008F75D5FF30200221C4854C92854D93D27E
:1009D0002043E68022203817C2AF53F2DFC296438D
:1009E000F24075D5EF43F210D2AF759F5341F9C273
:1009F000AF53F2DFC29443F21075D5BF43F240D239
:100A0000AF759F5341F9203817C2AF53F2EF75D538
:100A1000DF43F220C29643F240D2AF759F6341F9A3
:100A2000C2AF53F2BF75D5DF43F220C29443F21038
:100A3000D2AF759F2341F9203817C2AF53F2BFC21E
:100A40009443F21075D5DF43F220D2AF759F234156
:100A5000F9C2AF53F2EFC29643F24075D5DF43F2CD
:100A600020D2AF759F6341F9203817C2AF53F2DF30
:100A700075D5BF43F240C29443F210D2AF759F5375
:100A80008077C2AF53F2DF75D5EF43F210C29643C1
:100A9000F240D2AF759F538060203817C2AF53F237
:100AA000EFC29543F22075D5BF43F240D2AF759F98
:100AB000638046C2AF53F2BFC29543F22075D5EFB3
:100AC00043F210D2AF759F23802F203817C2AF5347
:100AD000F2BF75D5EF43F210C29543F220D2AF7545
:100AE0009F238015C2AF53F2EF75D5BF43F240C2CA
:100AF0009543F220D2AF759F63227A147B788012DF
:100B00007A107B8C800C7A0D7BB480067A0B7BC8C4
:100B10008000E564D5E001227902E453F2DFD5E0FC
:100B2000FDD29543F220D5E0FD53F2DFD5E0FDC2C2
:100B30009543F220D5E0FDE920E005D29643F2404E
:100B400030E005D29443F210E564D5E0FDE920E001
:100B50000353F2BF30E00353F2EF7496D5E0FDD9B2
:100B6000B9EAF8D5E0FDD8FBDBA853F2DF2253F257
:100B70008F53F28F75D5FF22788076FF0876FF08B5
:100B800076FF0876FF0876FF0876FF087609087674
:100B9000FF087601788C76010876FF0876FF0876E4
:100BA000FF0876FF0876FF0876030876FF0876FFD1
:100BB0000876FF0876250876D0087628087650084B
:100BC00076040876FF0876020876FF08767A0876BB
:100BD000FF0876070876010876FF0876FF0876009A
:100BE00008760022FA75F00CA4ABF0EAC333F8746F
:100BF0000133F9E8C333F8E933F9E8C32BF8E934F2
:100C000000F9227888E6C39403D23A5002C23AC26D
:100C100038E630E102D238A23892397886E614906C
:100C200000809378A6F67886E6F53FC394025003D9
:100C3000753F02789CE6753EFFB40203753EA0B492
:100C40000303753E8278A0E6F8600674282409D86C
:100C5000FCF5697896E671E488318932789EE67110
:100C6000E4883389347897E671E488358936716E83
:100C7000223036117A007B007CFF7D007E0091D708
:100C80008B618A6022303A227896E6FA7B00789E61
:100C9000E6FC7D00C3EA33FAEB33FBC3EC33FCED37
:100CA00033FD7E0A91D78B638A627896303A027858
:100CB0009EE6FA7B007897E6FC7D007E00303A10D5
:100CC000C3EA33FAEB33FBC3EC33FCED33FD7E0AAE
:100CD00091D78B618A6022C3EC9EFCED9400FDC32A
:100CE000EC9AFCED9BFDC3EC9423ED940050047C46
:100CF000237D00C3EC94FFED940140047CFF7D0153
:100D00007BFF0B7A000AEA7009C3EC33FCED33FD7C
:100D1000A102EC8AF0A4AEF0ED8AF0A42E947C40FF
:100D2000E4EAF460DD22D236917112054A12054AD6
:100D30007A007B007C10120542E5542AFA74003BCD
:100D4000FBDCF37C04C3EB13FBEA13FADCF7FFEBE9
:100D500060027FFFC23691712278A5E6F9540370D4
:100D600000E9540C7000E954307000E954C0700080
:100D7000227567007568007597DE7597AD7581C03F
:100D800043FF8075EF0675A900716E7580FF75F1E0
:100D90009375A4007580FF75D4FF75900075F28F70
:100DA00075A57075900075D5FF75A60175E3407542
:100DB000E202716EE4F8F6D8FD71781213CF7898DC
:100DC0008664753001C2AF12055251FA12054A719C
:100DD0000012054A710612054AB159C2AF75670083
:100DE00075680078FA79FA308707D9FBD8F7021CC2
:100DF000009103917178988664716E75E407758827
:100E000011758E0475890975C80475910475D840EB
:100E100075D90875F782759E0075960075DA4A7562
:100E2000DB0075A82175E69075B801759B80759DEE
:100E30000075D10C75BC5975BB1075E88075B20191
:100E400012053ED2AF753C00C230120552C231C20B
:100E500032C233C234755200755300752200120538
:100E60004EC3E522940A5002E132D23175220012BB
:100E7000054EC3E522940A5002E132C231D23275E6
:100E8000220012054EC3E522940A5002E13275E4B5
:100E9000F7758851758E017589AA758C00758D005E
:100EA000C2A9D2ABD2AA756BC0756A14756E50C256
:100EB00032D23475220A12054E756A10C3E52294A7
:100EC0000A7552007553004069758E0C756B8075FC
:100ED0006A28756E2875220A12054E756A20C3E5C8
:100EE00022940A7552007553004047758E0C756B3D
:100EF000C0756A14756E1475220A12054E756A1053
:100F0000C3E522940A755200755300402575E40725
:100F1000758811758E04758909D2A9C2ABC2AAC29F
:100F200034D23375220012054EC3E522940A4002E2
:100F3000A1DB120542203003020DDBC2AF51FA5192
:100F4000FA51FAD2AF120552203403303A03020F9D
:100F5000F0120542788CE6C394015002E1F0E530CE
:100F6000C394015002E1F07567A57568F17F02D264
:100F700036917112054EC2AFC2369171C3E55494D9
:100F80007FD2AF406B12053EC2AF710CD2AFDFDF34
:100F9000B126C3EF7897F61205521214BC7F0AD21D
:100FA00036917112054EC2AFC2369171C3E55494A9
:100FB0007FD2AF50E812053EC2AF51FA120546513A
:100FC000FAD2AFDFDAB126EF24037896F6F87997F4
:100FD000E7C394234003985006E824237897F61239
:100FE00005521214161214EB12054E9171020DDB0C
:100FF00075670075680012054EC3E55494014003FF
:10100000020F48C2AF120B0C120B0C120B0CD2AF1A
:10101000120552753000E4F537F5380537E537F439
:10102000703F0538789AE6781914601278321460A7
:101030000D787D14600878FA146003753800C3E5F4
:101040003898401D120B6E12053E15387537007822
:10105000998664C2AF120B0CD2AF789886641205E1
:101060004E120546E5237003020DDBC3E5549401DF
:10107000500AC3E5529401501602101B12054EE5AA
:10108000237003020DDB755200755300021231C349
:10109000E55294017017C2AF120B6E7899866412F4
:1010A0000AFA78988664D2AF12054E4123C3E552FE
:1010B00094027017C2AF120B6E78998664120B00FF
:1010C00078988664D2AF12054E4123C3E55294034B
:1010D0007017C2AF120B6E78998664120B0678985F
:1010E0008664D2AF12054E4123C3E55294047017B3
:1010F000C2AF120B6E78998664120B0C78988664D6
:10110000D2AF12054E4123C3E55294057017C2AF0A
:10111000120B6E78998664120B0C78988664D2AFA5
:1011200012054E4123C3E55294077019C3E5539449
:10113000065002016B7401303A0274037888F6C2DB
:1011400038C2394123C3E55294087019C3E553945A
:10115000065002016B7402303A0274047888F6D2A9
:1011600038D2394123C3E55294097017C3E553942B
:10117000065002016B303A0BC37888E69402F6C23F
:101180003A4123C3E552940A7016C3E553940650BE
:1011900002016B203A0A7888E62402F6D23A41230B
:1011A000C3E55294147025C3E55394065002016BB5
:1011B000C2AF901A0B740093D2AF7888F613C2387E
:1011C000C2394002D2384002D2398057C3E5529426
:1011D000157038C3E5539406404FC2AF901A0B7494
:1011E0000093D2AFF8B801027402B802027401B8D9
:1011F00003027404B8040274037888F613C238C278
:10120000394002D2384002D2398018C3E552940CDA
:1012100070117567A57568F1C3E5539406400A918E
:1012200016D2AF75520075530075670075680001DE
:101230006BC2AF120B6EE4D2AFE4F55EF524F52578
:10124000F53D755E0812053E1205A730EDFDA8BDFF
:10125000A9BEE97001F8885F1205AB755E08C2AFE0
:10126000120612855D5B855D5CD2AF303A07C238ED
:10127000303502D238D228753900120A99120ACABA
:101280001206211206281206211206281206211221
:10129000089F1209901209D512062812088F202CD7
:1012A00003120561302C03120591120990120A06EF
:1012B00012062812089F120990120A3712062812E5
:1012C000088F120990120A6812062812089F120944
:1012D00090120A991206281205A712088F12099077
:1012E000120ACA1205AB120628302827855D5B79E1
:1012F000187A0CC3E53999400EC228D2298A3B8559
:101300005D5B855D5C800CC3E55494014003021273
:101310008F619930291F202B1CE53B147006C229D0
:10132000D22A418FF53B203A07C3E554940140038C
:1013300002128F8064753C00203A0F78FA79A4E796
:1013400060027803C3E55598504FE523604B303A6F
:1013500017203805203507800F303502800A202BF2
:1013600007D22B855D5B41BF78F0302B05855D5B37
:101370007820C3E54898500302128F302B1BC22BF4
:10138000C238303502D238D229753B12855D5B41B7
:101390008F053CE5546002619C753C00C2AF120BA6
:1013A0006E752400752500D2AF12054E120B6E78B3
:1013B000A4E6600FC29643F240C29543F220C29465
:1013C00043F210C3E53C94044003020DDB01169088
:1013D0001A0D7820914FE520B4550AA3914FE520CE
:1013E000B4AA0280137567A57568F1120B7891167F
:1013F000756700756800801D901A0378807B0A91DC
:101400004FA308DBFA901A0F788C7B1A914FA30830
:10141000DBFA901A2922C2AF9192916F901A007450
:10142000109154A374079154A374219154901A03FA
:1014300078807B0A9153A308DBFA901A0F788C7B93
:101440001A9153A308DBFA91A59183901A2922E4FB
:1014500093F622E6438F01538FFDFFC3E583941C6F
:10146000400122EF8567B78568B7F0538FFE2243AE
:101470008F02438F018567B78568B7901A0DF053C7
:101480008FFC22901A0D74559154901A0E74AA91E3
:1014900054227A3079D07820901A40914FE520F785
:1014A00009A3DAF7227A3079D0901A40E7915409EB
:1014B000A3DAF9227C05120552DCFB22C2AF120A24
:1014C000FA120B00120B06120B0C120546120AFA46
:1014D000120B00120B06120B0C120546120AFA121E
:1014E0000B00120B06120B0CD2AF22C2AF120B0C68
:1014F000120B06120B00120AFA120546120B0C12FE
:101500000B06120B00120AFA120546120B0C120BF4
:0A15100006120B00120AFAD2AF22F5
:1019FD00020D71100721FFFFFFFFFFFF09FF01FF20
:101A0D0055AA01FFFFFFFFFF03FFFFFF25D0285061
:0D1A1D0004FF02FF7AFF0701FFFF0000FF3A
:101A400023575F4C5F30302320202020202020208F
:101A500023424C48454C492445464D3842313023B9
:101A60002020202020202020202020202020202076
:101C0000C2AFC2D37597DE7597AD7581C075A90057
:101C100043FF80752438752503B1DB7529A5752A26
:101C2000F143F18053A47FD28775D4FF75E3407DE3
:101C3000FA780379E67C10752200752300901DE880
:101C40007B06752498752501308702814820870816
:101C5000D8FBD9F9DCF781BA308708D8FBD9F9DC91
:101C6000F781BAB19BE493A3C39A6004DDC381BA40
:101C7000DBDBB18D600281317B08E493FAA3B16EA6
:101C8000DBF87A30B16E752200752300B18DEAFC65
:101C9000EBFDC3ED94FE400EB18D8A278B28ED300D
:101CA000E0048A828B83B18D7AC270D8C3ED94FE32
:101CB000601950CEBD0029EC600F7520007521FF22
:101CC000752900752A000200008100A827A92808AC
:101CD00009D804D90281DDB191EAF281D10D81A642
:101CE000C3ED94035051EDA2E092007AC5C3E582A2
:101CF0009400E583941C508C200010438F02438F86
:101D0000018529B7852AB7F0300027A827A9280818
:101D100009438F01538FFDD804D902A132C3E58353
:101D2000941C4003A3A117E28529B7852AB7F0A325
:101D3000A117538FFC81827AC1BD030CE493A3FAEF
:101D4000B152DCF8B14A81828184AA22AB23B16E00
:101D5000EBFAEA6222752608C3E52313F523E52290
:101D600013F52250066323A0632201D526EAB1DBD6
:101D7000B1DB75260AEAF4200102D287300102C2E3
:101D800087B1DBC3134002C201D526EB22B191EA31
:101D9000FB208702A191308702A196752608AE2408
:101DA000AF25C3EF13FFEE13FEB1DFB1DBC3EA13C0
:101DB0003087024480FA30E703632201C3E523132E
:101DC000F523E52213F52250066323A0632201D5F3
:101DD00026D9E52265236523F52222AE24AF250E00
:101DE0000FDEFEDFFCD20122424C48656C693437BD
:061DF0003164E8B10601B8
:00000001FF
